:020000020000FC
:0400000020C018956F
:0200060018954B
:02000C00189545
:0200120018953F
:1000160018951895189528432920576F6C666761BF
:100026006E672044756E637A6577736B69207777A0
:10003600772E646D7834796F752E646504E00EBF93
:100046000FE50DBFD1E0C0E07CD1909AA598AD9A9E
:10005600A498AC9AA398AB9AA198A99AA298AA9A9E
:10006600899A919A8D98959A8E98969AB898C09AE8
:100076008F98979ABA98C29AB998C19ABB98C39A18
:10008600BC98C49ABD98C59A5FEF8EEFE0E0F1E0A8
:1000960000E00193E130E9F7F330D9F7EFEFF0E054
:1000A6005BD15AD100E0999B0F5F9A9B0E5F10E0DF
:1000B60020E0003061F012E524E9013041F015EA54
:1000C60028E2023021F01FEF2EEF033001F00DD1B0
:1000D600919807FF919A1F2F133007FD919A202FB1
:1000E600919826FF919A08F0E62F26FD919A3BB14A
:1000F600919825FF919A08F0F72F25FD919A2F3FA9
:10010600919824FF919A09F4282F24FD919A0000D2
:10011600919823FF919A019123FD919A37FB91982B
:1001260022FF919A509F22FD919A000E919821FFED
:10013600919A08F4139421FD919A012D919820FF2C
:10014600919A1330A9F020FD919A16F634FB4CB122
:100156003EF0C23019F4D33009F4BACF4993B8CF80
:10016600403019F4D0E0CEEFB3CFD3E0C2E0B0CF49
:10017600919A1DECA62FB72F9C9911975C919D9B88
:100186005FEF0F930F910F930F910F930F913BB169
:1001960037FF15C034FB4CB156F0C23019F4D330DA
:1001A60009F40DC049930BC0D3E0C2E008C040304B
:1001B60019F4D0E0CEEF03C0D3E0C2E077C01A95C1
:1001C60001F774C0919A07FF91981F2F133007FD0E
:1001D6009198202F919A26FF919808F0E62F26FDF8
:1001E60091980000919A25FF919808F0F72F25FD28
:1001F60091980000919A24FF9198019124FD91987D
:100206003BB1919A23FF9198509F23FD9198000E40
:10021600919A22FF919808F4139422FD919837FB46
:10022600919A21FF91980000000021FD9198012DDF
:10023600919A20FF91981330A9F020FD919816F617
:1002460034FB4CB13EF0C23019F4D33009F4BACFC6
:100256004993B8CF403019F4D0E0CEEFB3CFD3E016
:10026600C2E0B0CF919810E4A62FB72F9C991197B2
:100276005C919D9B5FEF3BB137FF15C034FB4CB1E2
:1002860056F0C23019F4D33009F40DC049930BC0AF
:10029600D3E0C2E008C0403019F4D0E0CEEF03C08E
:1002A600D3E0C2E003C01A9531F700C0B0E0A0E089
:1002B600859BA160869BA260B09BA460879BA8607B
:1002C600B29BA061B19BA062B39BA064B49BA068E3
:1002D600B59BB1606FEF70E088949C9B6150704055
:1002E6006A0F7B1F9B9B6ECFF3CE38E04AEA0FEF77
:1002F600001F919808F0919A3A95377008F4919AF0
:10030600B9F7012F001F919808F0919A3A95377026
:1003160008F4919AB9F7022F001F919808F0919A64
:100326003A95377008F4919AB9F74A9501F73FEF75
:100336004FEF0000000000004A95D9F73A95C9F73B
:10034600089500E000BD01E009B900E00BB900E145
:100356000AB906E800BD08950FEF03D00A95E9F73C
:1003660008950F9300E50DD00A950000E1F70F916F
:1003760008950F9308E005D00A950000E1F70F9164
:1003860008950F9305E10A950000E9F700000F9123
:10039600089528432920576F6C6667616E6720446D
:1003A600756E637A6577736B69207777772E646DE0
:0803B6007834796F752E64653F
:00000001FF
